:03000000023905BD
:0C39050078FFE4F6D8FD75817102394CA2
:100EE50020000A3C2E2E2E3E004950436F6E6E6543
:100EF50063745245510A004950436F6E6E656374C1
:100F0500000A49504E6F41434B210A003E432C567F
:100F15002C43432CC0E4E0EFF2E5F020D1E8EDEA04
:100F2500EEEC49500A003E432C4D41432C2530320E
:100F350062583A25303262583A25303262583A259D
:100F4500303262583A25303262583A25303262588A
:100F55002C4D414320E0E4F0E5F10A003E432C56D8
:100F650045522C20332E3220EEF220257320257396
:100F75002CC2E5F0F1E8FF20495020ECEEE4F3EB5C
:100F8500FF0A004E6F762030332032303038003182
:100F9500303A32333A3230003E432C4C442C5052D6
:100FA5004F473A20202020202020202020202020CC
:100FB500202020202020202020202020202020202C
:100FC500202020202020202020202020202020201C
:100FD500202020202020202020202020202020200C
:100FE50020202020202020202CC4E0F2E020EFF05B
:100FF500EEF8E8E2EAE828F4E0E9EB290A003E2AFF
:101005002C312CCEF1EDEEE2EDFBE520EFE0F0E04A
:10101500ECE5F2F0FB20F1E5F2E5E2EEE3EE20E8A7
:10102500EDF2E5F0F4E5E9F1E00A003E412C41304E
:10103500312C2562752E2562752E2562752E256249
:10104500752C495020E0E4F0E5F120E0E4E0EFF212
:10105500E5F0E00A003E412C4130322C2562752E28
:101065002562752E2562752E2562752C495020E066
:10107500E4F0E5F120EEF1ED2E20F1E5F0E2E5F00A
:10108500E00A003E412C4130332C2562752E256245
:10109500752E2562752E2562752C495020E0E4F0E9
:1010A500E5F120F0E5E72E20F1E5F0E2E5F0E00AD4
:1010B500003E412C4130342C2562752E2562752E5B
:1010C5002562752E2562752CCCE0F1EAE020F1E56C
:1010D500F2E80A003E412C4130352C2562752E255B
:1010E50062752E2562752E2562752CD8EBFEE70AF2
:1010F500003E2A2C312CC4EEEF2E20EFE0F0E0EC80
:10110500E5F2F0FB20F1E5F2E5E2EEE3EE20E8EDB5
:10111500F2E5F0F4E5E9F1E00A003E422C53303106
:101125002C2562752CC6E4E0F2FC20E7E0EFF0EE3A
:10113500F1E020F1EEE5E4E8EDE5EDE8FF20EEF283
:1011450020F1E5F0E2E5F0E00A003E422C533032B2
:101155002C2562752CCEE1ECE5ED20F120F1E5F0D2
:10116500E2E5F0EEEC20E1E5E720EAE2E8F2E0ED89
:10117500F6E8E90A003E422C5330332C2562752CE3
:10118500CFE5F0E5E7E0EFF3F1EA20EFF0E820EF57
:10119500EEF2E5F0E520F1E2FFE7E820F120F1E5E8
:1011A500F0E2E5F0EEEC0A003E422C5330352C25FA
:1011B50062752CCAE0EDE0EB20F8E8F0EEEAEEE22D
:1011C500E5F8E0F2E5EBFCEDEEE3EE20EEE1ECE533
:1011D500EDE00A003E532C5330362C253032625850
:1011E5002530326258253032625825303262582512
:1011F5003032625825303262582C4D414320E0E4AC
:10120500F0E5F120F8E8F0EEEAEEE2E5F8E0F2E5E7
:10121500EBFCEDEEE3EE20EEE1ECE5EDE00A003E61
:10122500454E440A000A44756D7058202020202040
:1012350030302030312030322030332030342030EF
:1012450035203036203037203038203039203041B5
:1012550020304220304320304420304520304600A5
:101265000A3A003A20000A000A44756D70442020AD
:1012750020202030302030312030322030332030D3
:101285003420303520303620303720303820303982
:10129500203041203042203043203044203045204A
:1012A500304600457272206B657900526420656591
:1012B50070726F6D0A005264204D454D0A005264EC
:1012C50020436F64650A00577269746520436F6433
:1012D500650A0044656275674950204F4E0A00440F
:1012E500656275674950204F46460A004465627538
:1012F5006755736572204F6E0A00446562756755C0
:10130500736572204F46460A0044656275674D73E2
:1013150067204F6E0A0044656275674D7367204FFD
:1013250046460A00436F6E666967206C6F636B21E2
:101335000A00577220656570726F6D0A002053614F
:10134500766520656570726F6D210A0045727220A1
:101355004D414321004C6F61643E3E002A003C41F3
:1013650030313D003C4130323D003C4130333D00A1
:101375003C4130343D003C4130353D003C21003C92
:101385005330313D003C5330323D003C5330333D0A
:0D139500003C5330353D003C5330363D00E8
:06432800010B0001090079
:1042EB00C28E438910758BFF758DB7D2ABD28E22E0
:03001B0002387533
:10387500C0E0C083C082C0D0C28E758BFF758DB786
:1038850020060675A61E75A6E10509D202E50B60A0
:1038950002050BE50AD394014002150A050EE50E53
:1038A500540F7048D20EE50E543F7012D200907737
:1038B50056E0600A04F0E0D394B44002D206907753
:1038C50051E0600204F09071CFE0600214F090774F
:1038D50057E0D394014003E014F0300502050CE5F0
:1038E5000DD394644004D2068002050DE508D394F7
:1038F5000140021508D28ED0D0D082D083D0E032DC
:10088500C291C290D2B5C20B7D027C007F07124295
:10089500B48F25E525646060097D017F6012424FB4
:1008A500D20BE4FDFC7F0B1242B48F25E52530E623
:1008B500097D04E4FF124273D20B7D017C007F07A2
:1008C5001242B48F25E5257008FD7FFF12424FD2F5
:1008D5000B300B03126000C288C2A8C2AA7589003A
:1008E500123CB1907409E0B4FA06A3E064CE607BD3
:1008F500E4F52574012525F582E43474F583E4F0E7
:100905000525E525B443EC90740974FAF0A374CE7B
:10091500F0A374CCF090740F740AF0E4A3F0A30470
:10092500F0A3F090740574FFF0A3F0A3F0E4A3F036
:10093500907420740AF0E4F525E5252401FFE433DD
:10094500FE74012525F582E43474F583E0FD124239
:100955002B0525E525C3944340DFE4F5A775A61EC1
:1009650075A6E1907FF0F0A3F080FE9074147403F7
:10097500F0A374CCF0E4907413F012338FC2B51267
:100985003681C206123F9FD20BC20DC20C90764132
:100995007408F090737F7424F0E4A3F0907409E078
:1009A500907381F090740AE0907382F090740BE07C
:1009B500907383F090740CE0907384F090740DE064
:1009C500907385F090740EE0907386F0750A01E4DB
:1009D500907642F0C207C208C209C20A1242042038
:1009E5000B19AF257E007D031232AEE4FF1235D11F
:1009F5007E0E7FE5E4FBFDFC122ED2907756E0607B
:100A0500037401F0E49071CFF0F50C907640F0F5A9
:100A15000D1242EB75A70775A61E75A6E1D2AFE4C8
:100A2500F50D9071CFE07003121B75907757E0B408
:100A350001119080007410F0E4907757F0D20BC24A
:100A45000CC20D908008E0F52530E405D20774103E
:100A5500F0E52530E508D2099080087420F0E525F9
:100A650030E608D2089080087440F0E50CC3940382
:100A75004019908002E4F0908001F0908000F0E54C
:100A85000C94064006E4F50C123F9F9080A0E070A0
:100A950003123D2F9080B8E07003123DA99080D0DD
:100AA500E07003123F43908000E07013300710128E
:100AB5002FD99073FCEFF0D39400400312002690D9
:100AC5008002E07006908000E06005D205020A24ED
:100AD500C205E4F50C9071CFE06003020A24200BF7
:100AE50012907643E0600C7E0E7FE71231C6E490EB
:100AF5007643F0300912122ADC9073FCEFF0D394A0
:100B0500004005E0FF1242FB200803020C8D12296C
:100B1500559073FCEFF07003020A24907440E05482
:100B2500BF247F7003020BF6147003020BCE240260
:100B35006003020C2F200B077E0E7FEE1231C620BC
:100B45000F03020C8D907418E0700690741CE06021
:100B55006790774DE0FF907418E0B5072490774EC5
:100B6500E0FE907419E0B5061890774FE0FE90749A
:100B75001AE0B5060C907750E0FE90741BE06E60AD
:100B85003790741CE06F6003020C8D90774EE0FF88
:100B950090741DE06F6003020C8D90774FE0FF901D
:100BA500741EE06F6003020C8D907750E0FF907427
:100BB5001FE06F6003020C8DC2039076427401F052
:100BC500120021750A01020C8D907756E0600374BE
:100BD50001F0907745E0FF907442E06F6003020CEE
:100BE5008D907745E004F0E4F50A907640F0020C2C
:100BF5008D300303020C8D90740FE07003020A24FC
:100C0500907420740AF012432FD203E4F50A90760B
:100C150040F090775104F0E4907744F0A3F0200B76
:100C2500677E0E7FFC1231C6805E907756E06003CA
:100C35007401F0300352907440E020E74B90744209
:100C4500E0FF907744E0FE6F600D90774CE0700711
:100C5500EE146F70338013907744E004F09073FCCA
:100C6500E0FFD3940440031240D19070CB7482F01E
:100C7500A37401F0907442E09070CDF07E707FCB4C
:100C85007D03123A18020A24200303020DA5E50A82
:100C9500706812417BEF60237E757F40907541E05F
:100CA5002404FD123A1890774CE07009907420E006
:100CB500F50A020A24E4F50A020A24907751E0D3E2
:100CC500943C403690774CE0703090775104F012A8
:100CD5004315E4907540F0A37412F0907745E090C9
:100CE5007542F0A374FDF09071D063A20190754434
:100CF50063A2017F121224D9809E12430A8F25E533
:100D050025B401159070CB7483F0E4A3F07E707F59
:100D1500CB7D02123A18020A24E525D39401401C22
:100D25009070CB7483F0A37401F0E52524FEA3F045
:100D35007E707FCB7D03123A18020A24E50A64010E
:100D45006003020A24907640E004F0200B077E0F32
:100D55007F061231C6907420E0C394C85004E02485
:100D650032F0907640E0C39405400DC203E49076DE
:100D750042F0120021020A247C777D4D907414E024
:100D8500FAA3E0FB7F02123BA97E757F4090754177
:100D9500E02404FD123A18907420E0F50A020A24B2
:100DA500E50A64016003020A24907642E014604675
:100DB50024FE6042147003020E9824046003020AA4
:100DC50024E4F50C200F139076427404F0907640DD
:100DD500E05401F0750A01020A249080027410F0B3
:100DE500E4907642F090764004F0750AFA90774DDB
:100DF50074FFF0020A2490774DE07003020E829092
:100E050075407480F09075427401F0E4A3F0A3047A
:100E1500F0A37430F0A3747BF0E4F5257447252521
:100E2500F582E43475F583747DF074482525F582E3
:100E3500E43475F583E4F0E5252407907541F07CED
:100E4500777D4D907414E0FAA3E0FB7F02123BA975
:100E55007E757F40E5252409FD123A1890774CE010
:100E6500601B12432FD203E4F50A907640F0907789
:100E75005104F0E4907744F0A3F0020A24300F0700
:100E8500E4907642F080069076427404F0750AFA92
:100E9500020A249080027410F0750A05907640E0ED
:100EA5006401FFF09076427401F0EF701990741CA4
:100EB500E06013FCA3E0FDA3E0FEA3E0FF90774D07
:100EC50012226E020A24907418E0FCA3E0FDA3E050
:0F0ED500FEA3E0FF90774D12226E020A2480FEEA
:010EE40022EB
:10002600907441E0B444047F0180027F00907440E4
:10003600E0B447047E0180027E00EE5F604A907461
:1000460009E0907442F090740AE0907443F0907462
:100056000BE0907444F090740CE0907445F090744A
:100066000DE0907446F090740EE0907447F0907432
:10007600417452F090737963A2019080A863A20143
:100086007F061224D902087B9073FCE0C3940850C3
:1000960003020884907409E0FF907442E06F6003E5
:1000A60002088490740AE0FF907443E06F600302D4
:1000B600088490740BE0FF907444E06F60030208BC
:1000C6008490740CE0FF907445E06F60030208842E
:1000D60090740DE0FF907446E06F60030208849010
:1000E600740EE0FF907447E06F600302088490741A
:1000F60041E0B44415907379E0B4FF0E63A2019019
:1001060080A863A2017F061224D9907756E0600387
:100116007401F09077577464F09074417452F090C3
:100126007440E0646D60030202857BFF7A0F7911EB
:1001360012187B7BFF7A0F792B907409E0F52EA3BA
:10014600E0F52FA3E0F530A3E0F531A3E0F532A307
:10015600E0F53312187B752EFF752F0F75308875F5
:1001660031FF75320F7533947BFF7A0F7961121860
:100176007B7BFF7A0F799D12187B7BFF7A107903C0
:1001860012187B7BFF7A10793090740FE0F52EA35E
:10019600E0F52FA3E0F530A3E0F53112187B7BFFE5
:1001A6007A10795A907418E0F52EA3E0F52FA3E0A3
:1001B600F530A3E0F53112187B7BFF7A1079889031
:1001C600741CE0F52EA3E0F52FA3E0F530A3E0F5CF
:1001D6003112187B7BFF7A1079B6907405E0F52E04
:1001E600A3E0F52FA3E0F530A3E0F53112187B7BF1
:1001F600FF7A1079D9907401E0F52EA3E0F52FA3CC
:10020600E0F530A3E0F53112187B7BFF7A1079F622
:1002160012187B7BFF7A11791FA20FE433F52E1299
:10022600187B7BFF7A11794F90774CE0F52E1218E8
:100236007B7BFF7A11797A907756E0F52E12187B40
:100246007BFF7A1179ADA201E433F52E12187B7B80
:10025600FF7A1179D9907746E0F52EA3E0F52FA322
:10026600E0F530A3E0F531A3E0F532A3E0F5331273
:10027600187B12372F7BFF7A12792412187B229073
:100286007440E0644C70737E127F2AFBFDFC122ED4
:10029600D2907448E0F526A3E0F527E4F529E52693
:1002A60090744AF0A3E527F07E127F657C747D4A40
:1002B6007B02122ED2E4F528852782852683E0FF6D
:1002C600744A2528F582E43474F583EFF00527E5B2
:1002D60027700205260528E528B410DC7E127F6803
:1002E6007C747D4A7B10122ED20529E529C3941011
:1002F60040AC7E127F6B1231C622907440E0646C73
:100306007060F52A7E127F6DFBFDFC122ED2E4F59D
:1003160029E490744AF0A3E52AF07E127F657C7486
:100326007D4A7B02122ED2E4F528A82AE6FF744AFB
:100336002528F582E43474F583EFF0052A0528E5CF
:1003460028B410E67E127F687C747D4A7B10122EDC
:10035600D20529E529C3940840B77E127F6B123176
:10036600C622907440E0644B7061F52874322528EB
:10037600F582E43474F583E0603274322528F58220
:10038600E43474F583E0F4602374322528F582E4BE
:100396003474F583E0FF74482528F582E43474F557
:1003A60083E0B507100528E528B408C09071CF741E
:1003B60032F002087B9074407421F0300B0302087F
:1003C6007B7E127FA81231C602087B907440E0B48F
:1003D600521A200B077E127FB01231C690744074F9
:1003E60072F07E747F407D0812399122907440E04D
:1003F60064497045200B077E127FBB1231C690748C
:1004060048E0F526A3E0F527E4F52885278285262A
:1004160083E0FF744A2528F582E43474F583EFF00F
:100426000527E527700205260528E528B480DC7E29
:10043600747F407D8A12399122907440E064437043
:1004460046200B077E127FC31231C6907448E0F532
:1004560026A3E0F527E4F528852782852683E493FD
:10046600FF744A2528F582E43474F583EFF00527F6
:10047600E527700205260528E528B480DB7E747F13
:10048600407D8A12399122907440E0645A7053205C
:100496000B077E127FCC1231C6907448E0F526A376
:1004A600E0F5277C747D4A7B80AF27AE2612414754
:1004B600E4F528852782852683E493FF744A252858
:1004C600F582E43474F583EFF00527E5277002051D
:1004D600260528E528B480DB7E747F407D8A1239A4
:1004E6009122907440E06444600302057990744858
:1004F600E0FF6444700302087BEFB4310CC20B7E4C
:10050600127FD81231C602087B907448E0B4300CD2
:10051600D20B7E127FE41231C602087B907448E04B
:10052600B4320CD20C7E127FF11231C602087B90D7
:100536007448E0B4330CC20C7E127FFF1231C6023F
:10054600087B907448E0B4340CD20D7E137F0E12F3
:1005560031C602087B907448E0B4350CC20D7E1398
:100566007F1B1231C602087B907448E0FF12001E02
:1005760002087B9071CFE07013200B077E137F2952
:100586001231C69074407421F002087B9071CF74CA
:1005960032F0907440E0FFB45104C2AF80FEEF64C5
:1005A600577045200B077E137F371231C69074496A
:1005B600E09073FCF0E4F5289073FCE0FFE528C3B7
:1005C6009F400302087B744A2528F582E43474F5BB
:1005D60083E0FF907448E025282478F582E434729D
:1005E600F583EFF0052880D0907440E064536003F3
:1005F60002069C200B077E137F421231C6907409B7
:10060600E0FF907281E06F703C90740AE0FF907298
:1006160082E06F703090740BE0FF907283E0B50754
:100626002490740CE0FF907284E0B5071890740D66
:10063600E0FF907285E0B5070C90740EE0FF9072B3
:1006460086E06F60169074407421F0300B03020848
:100656007B7E137F511231C602087BE4F528E4F550
:100666000DAF28FE74782528F582E43472F583E010
:10067600FD12422B0528E528C394FE40E1C2AFE4F3
:10068600907FF0F0A3F0907FFD74AAF0A374FFF0C2
:10069600A37455F080FE907440E0644F704C9074E3
:1006A60048E0F526A3E0F527E5274526700A200B46
:1006B600077E137F5A1231C6200B077E137F611205
:1006C60031C6E4F528744A2528F582E43474F583A6
:1006D600E0852782852683F00527E5277002052613
:1006E6000528E528B480DE02087B907440E0FFB45C
:1006F6004521907448E0FDA3E0907FF0CDF0A3ED96
:10070600F0C2AF907FFD74AAF0A374FFF0A37455F6
:10071600F080FEEF64656003020884907448E0FF91
:10072600A3E0907FF0CFF0A3EFF0E4F526F527D312
:10073600907FF1E09527907FF0E095264020E4F544
:100746000D2527FFE5263401FE852782852683E0D1
:10075600FD12422B0527E5277002052680D17E1360
:100766007F63123A9FEF4E602012000390740FEFE2
:10077600F0120003907410EFF0120003907411EF62
:10078600F0120003907412EFF07E137F69123A9F05
:10079600EF4E6020120003907418EFF012000390E1
:1007A6007419EFF012000390741AEFF01200039020
:1007B600741BEFF07E137F6F123A9FEF4E6020128C
:1007C600000390741CEFF012000390741DEFF012FA
:1007D600000390741EEFF012000390741FEFF07E7A
:1007E600137F75123A9FEF4E602012000390740536
:1007F600EFF0120003907406EFF0120003907407F6
:10080600EFF0120003907408EFF07E137F7B123A2C
:100816009FEF4E6020120003907401EFF012000368
:10082600907402EFF0120003907403EFF0120003CD
:10083600907404EFF0E4F528E4F50DE5282401FFB3
:10084600E433FE74012528F582E43474F583E0FD73
:1008560012422B0528E528C3944340DCC2AFE4903E
:100866007FF0F0A3F0907FFD74AAF0A374FFF0A3CD
:0E0876007455F080FE7E747F407D081239912B
:010884002251
:10410F00AE07EEC39430400BEED394395005EE2436
:10411F00D0FF22EEC39461400BEED394665005EEB0
:10412F0024A9FF22EEC39441400BEED394465005D1
:08413F00EE24C9FF22AF0622A5
:1042D100907378E004F07006907377E004F09073C7
:0A42E10077E0FEA3E0FF12429722EF
:100003001242D112410FEFC454F0FEC0061242D186
:0800130012410FD0E02FFF2283
:103EE600E49078B0F01242D19078B1EFF0C39430FC
:103EF6004018E0FFD3943950119078B0E024D0F503
:103F060082E43471F583EFF080119078B0E024D02C
:103F1600F582E43471F583E4F0800C9078B0E00427
:103F2600F0E0D3940840BE752900752A00752B0071
:0C3F3600E4F52C7B017A7179D01227B1E0
:013F4200225C
:043A9F008E2B8F2CAF
:103AA300907377E4F0A374FFF01242D1EF606EF4E9
:103AB300606B852C82852B83E493B507EC752D0110
:103AC300E52C252DF582E4352BF583E493602590D1
:103AD3007378E0252DFF907377E03400FE12429750
:103AE300E52C252DF582E4352BF583E493B5070406
:103AF300052D80CCE52C252DF582E4352BF583E4CB
:103B03009370A6E52D24FFFFE434FFFE907378E065
:103B13002FF0907377E03EF07E007F0122E4FEFFFA
:013B2300227F
:10338F007E137F81123A9FEF4E70037F01227E13CF
:10339F007F84123A9FEF4E600C1242D1EF24D0245B
:1033AF00FF920F8002D20F7E137F8A123A9FEF4E49
:1033BF00600C1242D1EF24D090774CF08005E4904E
:1033CF00774CF07E137F90123A9FEF4E600C1242B3
:1033DF00D1EF24D0907756F08005E4907756F07EA9
:1033EF00137F96123A9FEF4E600C1242D1EF24D00A
:1033FF0024FF92018002C20190740963A2019077A9
:10340F004663A2017F061224D930013B7E137F9CB5
:10341F00123A9FEF4E6030120003907746EFF01292
:10342F000003907747EFF0120003907748EFF01208
:10343F000003907749EFF012000390774AEFF012F4
:0A344F00000390774BEFF07F00229E
:10404300907641E0C3947C503D907641E0FE04F0CD
:10405300747F2EF582E43473F583EFF0BF0A279063
:104063007641E0FF04F0747F2FF582E43473F58327
:10407300E4F0907641E0FF123B249076417408F01F
:07408300907380E004F022BD
:103F9F009080007480F090740163A201F583F58224
:103FAF0063A2017F081224D990740963A201908043
:103FBF008863A2017F0A1224D9908092E4F0A3743F
:103FCF0032F0A37401F0907413E0FF9080B1F09081
:103FDF0080E1EFF09080957455F0A3F0908000741D
:093FEF0001F090800974F0F02249
:103D2F00908009E04410F09080A0E0706C9080A12A
:103D3F007482F09080A874FFF0A3F0A3F0A3F07F3B
:103D4F00039080AEEFF07FCBA3EFF07F039080ACBA
:103D5F00EFF0A374CBF09080007402F09078A4126F
:103D6F00227A000000009078A4E0908040F09078D4
:103D7F00A5E0908041F09078A6E0908042F0907896
:103D8F00A7E0908043F0A3E4F0A3F0A3F0A3F0909A
:093D9F008018F0A3F0A3F0A3F0DA
:013DA80022F8
:103F4300908009E04440F09080D17482F07F039028
:103F530080DEEFF0A374CCF09080027402F09078CE
:103F6300A812227A000000009078A8E0908058F010
:103F73009078A9E0908059F09078AAE090805AF068
:103F83009078ABE090805BF0A3E4F0A3F0A3F0A300
:0B3F9300F0908030F0A3F0A3F0A3F04A
:013F9E002200
:103DA900908009E04420F09080B8E0706C9080B970
:103DB9007482F07F039080C6EFF07FCDA3EFF07F90
:103DC900039080C4EFF0A374CDF09080C074FFF02D
:103DD900A3F0A3F0A3F09080017402F09078AC12E4
:103DE900227A000000009078ACE090804CF0907846
:103DF900ADE090804DF09078AEE090804EF09078F4
:103E0900AFE090804FF0A3E4F0A3F0A3F0A3F0900B
:093E19008024F0A3F0A3F0A3F053
:013E2200227D
:103BA9008C268D27A907EAFDE975F018A424ACFF36
:103BB900E5F034808F82F583EDF0EBFDE975F018BF
:103BC900A4FFAEF024ACFBEE34808B82F583A3ED29
:103BD900F08527828C83E0FDEF24A8FFEE3480FE78
:103BE9008F82F583EDF08527828C83A3E08F828E07
:103BF90083A3F0852782852683A3A3E0FDE975F0D9
:103C090018A424A8FFE5F03480FE8F82F583A3A3CE
:103C1900EDF08527828C83A3A3A3E08F828E83A3F3
:043C2900A3A3F0223F
:063991008D2BAB07AA0616
:10399700908000E030E5079076437401F02290783C
:1039A700A4E0FCA3E0FDA3E0FEA3E0F52F8E2E8D9F
:1039B7002D8C2CAE02AF038E838F8263A201E52E7E
:1039C700540744C0F583852F8263A201AF2B1225CC
:1039D7004BE4FCFDFEE52F252BF52FEE352EF52EBE
:1039E700ED352DF52DEC352CF52C908040E52CF0A0
:1039F700A3E52DF0A3E52EF0A3E52FF0908000744A
:103A070020F0AF2FAE2EAD2DAC2C9078A412226EE5
:013A1700228C
:063A18008D26AB07AA0693
:103A1E00908002E030E5079076437403F0229078B0
:103A2E00A8E0FCA3E0FDA3E0FEA3E0F52A8E298D1D
:103A3E00288C27AE02AF038E838F8263A201E52905
:103A4E00540744D0F583852A8263A201AF2612253E
:103A5E004BE4FCFDFEE52A2526F52AEE3529F5294F
:103A6E00ED3528F528EC3527F527908058E527F019
:103A7E00A3E528F0A3E529F0A3E52AF090800274CF
:103A8E0020F0AF2AAE29AD28AC279078A812226E6E
:013A9E002205
:0235D1008F2742
:1035D300908001E030E5099076437402F07F002289
:1035E3009078ACE0FCA3E0FDA3E0FEA3E0F52B8E16
:1035F3002A8D298C2890774663A201E52A54074433
:10360300C8F583852B8263A2017F06122561E52B12
:103613002406F52BE4352AF52AE43529F529E43582
:1036230028F52890764463A201E52A540744C8F597
:1036330083852B8263A201AF27122561E4FCFDFE83
:10364300E52B2527F52BEE352AF52AED3529F52926
:10365300EC3528F52890804CE528F0A3E529F0A364
:10366300E52AF0A3E52BF09080017420F0AF2BAE98
:0D3673002AAD29AC289078AC12226EAF274A
:013680002227
:102FD9009081E0E0F5260526052605260526052625
:102FE90005260526052605260526908010E0F529E3
:102FF900A3E0F52AA3E0F52BA3E0F52C9081E1E00D
:10300900F52605260526052605260526052605266F
:10301900052605260526908014E0F52DA3E0F52E5A
:10302900A3E0F52FA3E0F530E52FB52B08E530B582
:103039002C037F0022E4F526E52F540744E0F583AD
:1030490085308263A20190744063A2017F08122532
:103059009190744263A20190737963A2017F061271
:1030690024D9907440E0F527A3E0F528E4F52690EB
:103079007440E0702AA3E024F8F526E52F540744AC
:10308900E0F58385308274082582F582E43583F57D
:103099008363A20190744063A201AF26122591AE09
:1030A90027E4FCFDE5302528F530E52F3EF52FED29
:1030B900352EF52EEC352DF52D908014E52DF0A348
:1030C900E52EF0A3E52FF0A3E530F09080007440E1
:0330D900F0AF262F
:0130DC0022D1
:102955009081E6E0F52605260526052605260526A9
:1029650005260526052605260526908028E0F52955
:10297500A3E0F52AA3E0F52BA3E0F52C9081E7E091
:10298500F5260526052605260526052605260526FA
:1029950005260526052690802CE0F52DA3E0F52ECD
:1029A500A3E0F52FA3E0F530E4F526E52FB52B0AD6
:1029B500E530B52C05C208022AC1E52F540744F0BD
:1029C500F58385308263A20190744063A2017F087C
:1029D500122591907440E0F527A3E0F528E52845F8
:1029E5002770099080027410F07F002290774DE0E7
:1029F500FFF46030907442E06F6003022A8890779C
:102A05004EE0FF907443E06F707990774FE0FF9050
:102A15007444E06F706D907750E0FF907445E06FFF
:102A25006031805F907442E090774DF0907443E0A0
:102A350090774EF0907444E090774FF0907445E0B5
:102A4500907750F0907446E0FFA3E0907414CFF0B7
:102A5500A3EFF0907440E0702AA3E024F8F526E592
:102A65002F540744F0F58385308274082582F5825A
:102A7500E43583F58363A20190744063A201AF2618
:102A8500122591AE27E4FCFDE5302528F530E52F2C
:102A95003EF52FED352EF52EEC352DF52DAF2CAE63
:102AA5002BAD2AAC29AB30AA2FA92EA82DD31222E3
:102AB5005D40099080027410F07F002290802CE523
:102AC5002DF0A3E52EF0A3E52FF0A3E530F09080DF
:062AD500027440F0AF2680
:012ADB0022D8
:102ADC009081E3E0F5260526052605260526052624
:102AEC000526052605260526052690801CE0F529D9
:102AFC00A3E0F52AA3E0F52BA3E0F52C9081E4E00C
:102B0C00F526052605260526052605260526052671
:102B1C00052605260526908020E0F52DA3E0F52E50
:102B2C00A3E0F52FA3E0F530E4F526E52FB52B0A4D
:102B3C00E530B52C05C209022C32E52F540744E8C8
:102B4C00F58385308263A2019070CF63A2017F0E62
:102B5C001225A79070CFE0F527A3E0F5289070D749
:102B6C00E0FFF4604A907746E0FEEF6E7079A3E0E8
:102B7C00FF9070D8E06F706F907748E0FF9070D93D
:102B8C00E06F7063907749E0FF9070DAE06F7057F8
:102B9C0090774AE0FF9070DBE06F704B90774BE0E2
:102BAC00FF9070DCE06F703FE49070DEF080089076
:102BBC0070DE74FFF0D2D99070CFE0702AA3E024BD
:102BCC00F2F526E52F540744E8F583853082740E20
:102BDC002582F582E43583F58363A2019070CF637F
:102BEC00A201AF261225A7AE27E4FCFDE53025286F
:102BFC00F530E52F3EF52FED352EF52EEC352DF578
:102C0C002DAF2CAE2BAD2AAC29AB30AA2FA92EA8F8
:102C1C002DD312225D5006E52845277009908001BE
:102C2C007410F07F0022908020E52DF0A3E52EF0AB
:102C3C00A3E52FF0A3E530F09080017440F0AF26AF
:012C4C002265
:0431C6008E2C8F2D8F
:1031CA00908000E030E5079076437401F022907811
:1031DA00A4E0FCA3E0FDA3E0FEA3E0F5338E328D6C
:1031EA00318C30E533FFE5325407FEE42FF52FEE3C
:1031FA0034C0F52E852F82F5837423F0052FE52F31
:10320A007002052E532EC7F582852E83740AF005A7
:10321A002FE52F7002052E532EC790740963A20161
:10322A00852E83852F8263A2017F0612254B7406A1
:10323A00252FF52FE4352EF52E852C83852D8263D7
:10324A00A201852E83852F8263A20112252FE4FC19
:10325A00FDFE9078A4E0F8A3E0F9A3E0FAA3E02F3A
:10326A00FFEE3AFEED39FDEC38FCEF2408FFE43EB0
:10327A00FEE43DFDE43CFC9078A412226E9078A412
:10328A00E0908040F09078A5E0908041F09078A698
:10329A00E0908042F09078A7E0908043F090800020
:0332AA007420F09D
:0132AD0022FE
:0A2ED2008E2B8F2C8C2D8D2E8B2F54
:102EDC00908000E030E5079076437401F022907802
:102EEC00A4E0FCA3E0FDA3E0FEA3E0F5358E348D59
:102EFC00338C32E535FFE5345407FEE42FF531EE23
:102F0C0034C0F530853182F5837423F00531E53119
:102F1C00700205305330C7F582853083740AF00592
:102F2C0031E531700205305330C790740963A2014A
:102F3C0085308385318263A2017F0612254B74068E
:102F4C002531F531E43530F530852B83852C8263C2
:102F5C00A20185308385318263A20112252F8F3621
:102F6C00EF2531F531E43530F530E52F6017852D3F
:102F7C0083852E8263A20185308385318263A20111
:102F8C00AF2F12254BE5362408252FF52FFFE4FC37
:102F9C00FDFEE5352FF535EE3534F534ED3533F5ED
:102FAC0033EC3532F532908040E532F0A3E533F066
:102FBC00A3E534F0A3E535F09080007420F0AF3534
:0C2FCC00AE34AD33AC329078A412226E0B
:012FD80022D6
:023B24008F3FD1
:103B2600908000E030E5079076437401F0229078AB
:103B3600A4E0FCA3E0FDA3E0FEA3E0F5438E428DE6
:103B4600418C40E543FFE5425407FEE42FFFEE3487
:103B5600C090737F63A201F5838F8263A201AF3F9A
:103B660012254BE4FCFDFEE543253FF543EE3542C9
:103B7600F542ED3541F541EC3540F540908040E5A4
:103B860040F0A3E541F0A3E542F0A3E543F09080C1
:103B9600007420F0AF43AE42AD41AC409078A41221
:023BA600226E8D
:013BA80022FA
:0632AE008E298F2AAB05FA
:1032B400908000E030E5079076437401F022907826
:1032C400A4E0FCA3E0FDA3E0FEA3E0F5308E2F8D87
:1032D4002E8C2DE530FFE52F5407FEE42FF52CEE60
:1032E40034C0F52B852C82F5837423F0052CE52C52
:1032F4007002052B532BC7F582852B83EBF0052C2D
:10330400E52C7002052B90740963A201852B83853B
:103314002C8263A2017F0612254B7406252CF52C02
:10332400E4352BF52B532BC7E529852C82852B837C
:10333400F0052CE52C7002052B532BC7F582852B49
:1033440083E52AF0052CE52C7002052B532BC7E5E9
:1033540030240AF530E4352FF52FE4352EF52EE42C
:10336400352DF52D908040E52DF0A3E52EF0A3E555
:103374002FF0A3E530F09080007420F0AF30AE2F32
:0A338400AD2EAC2D9078A412226E3D
:01338E00221C
:10429700A2AF9210C2AF438E2075D2028F828E8357
:0C42A700E0FFE4F5D2538EDFA21092AFCE
:0142B30022E8
:10422B00E5D220E0FBA2AF9210C2AF43D2028F8245
:10423B008E83EDF075D25063D250A21092AFE5D2BF
:03424B0020E0FB75
:01424E00224D
:103CB100E4FDED2401FFE433FE12429774012DF57A
:103CC10082E43474F583EFF00DBD3FE6E4FDED24AD
:103CD1007FFFE433FE12429774F82DF582E43471CC
:103CE100F583EFF074F82DF582E43471F583E0701B
:103CF1001B74F82DF582E43471F5837420F074F9A6
:103D01002DF582E43471F583E4F080040DBD80BEAD
:103D1100E4907277F0FDEDFF7E0012429774782DEA
:0D3D2100F582E43472F583EFF00DBDFEE98C
:013D2E002272
:024147008B2BC0
:10414900A2AF9210C2AF85A22C53A2FE8E838F829A
:1041590005A28C838D8274091225D5E52B53A2FE05
:1041690043A2201225D753A2DF852CA2A21092AF19
:01417900FF46
:01417A002222
:1042B400A2AF9210C2AF8C838D82EF1225D543A298
:0C42C400201225D753A2DFA21092AFFFFA
:0142D00022CB
:02424F008F26B8
:10425100A2AF9210C2AFE4F5838D8274061225D508
:10426100E52643A2201225D753A2DFA21092AF7FE9
:01427100014B
:014272002229
:024273008F2694
:10427500A2AF9210C2AFE4F5838D82740A1225D5E0
:10428500E52643A2201225D753A2DFA21092AF7FC5
:014295000127
:014296002205
:1023FE00A907E7FFA805EF93C3966008403B74FC5E
:10240E002FFF80F00F08EF93C3966008402B74FBEC
:10241E002FFF80E00F08EF93C3966008401B74FAFD
:10242E002FFF80D00F08EF93D3966008400B74F9FE
:10243E002FFF80C01F1F1F1F1FEF54FEF80303F74F
:10244E00E893FC08E893FD08E893FE08E893FF2262
:10245E0009E993C39D6008402974FB29F980F109AD
:10246E00E993C39E6008401A74FA29F980E209E9DB
:10247E0093D39F6008400B74F929F980D319191969
:10248E001919E9C313C313FF22740093F8ECC39810
:10249E004024701F740193F8EDC3984019701474A2
:0E24AE000293F8EEC398400E7009740393F881
:1024BC00EFC39840037F00227F0122EDF8E6F0087D
:1024CC00A3DFFA22EDF8E0F608A3DFFA22E0A3631B
:1024DC00A201F0A363A201DFF475A2002263A201A2
:1024EC00F0A363A20122E0A363A201F0A363A20103
:1024FC00E0A363A201F0A363A201E463A201F0A331
:10250C0063A201DFE175A20022E0A363A2016DFECC
:10251C00936CFDEE058393FC158363A201DFEA75D2
:10252C00A200227F00E493A363A201F00F600CA32E
:10253C00E583C2E3F58363A20180EA75A20022E081
:10254C00A363A201F0A3E583C2E3F58363A201DFD9
:10255C00EE75A20022E0A363A201F0A3E583C2E41E
:10256C00D2E3F58363A201DFEC75A20022E0A36342
:10257C00A201F0A3E58344F8C2E5F58363A201DF71
:10258C00EC75A20022E583C2E3F583E0A363A2010C
:10259C00F0A363A201DFEE75A20022E583C2E4D2B0
:0A25AC00E3F583E0A363A201F0A3AE
:1025B60063A201DFEC75A20022E58344F8F583E00F
:1025C600A363A201F0A363A201DFEE75A20022F9C4
:1025D60022C002C004C00612FFF0D006D004D0020A
:0125E60022D2
:1037D4004572724C656E210A000A496E49503A00DE
:1037E400205544502054696D654750530A00200AFF
:1037F400495054696D653A2000200A4441544147B8
:1038040052414D3A20002049676E6F72650A2000CC
:103814002043414E2054696D654750530A0020549B
:103824007261737353656E644552520A000ACEF88E
:10383400C4EBE8EDFB43414E210A000A4572724194
:10384400647243414E3A00205265496E69742043C4
:10385400414E0A002043414E283029203E20544F37
:10386400210A0020545520300A0020545520310AE2
:013874000053
:03001E00E4FF22DA
:1041DC00C2A9438902758C48758A4875D90475DB68
:1041EC004875DC4875DD4875DE48E4F5E9F5F9D22B
:0841FC00D9C2DAD28CD2DE2216
:1041AE00C2D990776CE07013E5E92419F5EB30D79E
:1041BE0006E5F904F5FB2285F9FB22E5E924C8F5AD
:0E41CE00EB30D706E5F904F5FB2285F9FB225C
:10408A00C2D990776CE0702C301D16E5E92432F520
:10409A00EB30D707E5F904F5FB800385F9FBC21D70
:1040AA0022E5E92405F5EB30D706E5F904F5FB220C
:1040BA0085F9FB22E5E92432F5EB30D706E5F90468
:0740CA00F5FB2285F9FB2242
:104204001241DC90776CE0C394645006123C2D128A
:1042140041AE120022D21CE4F56D907884F0F55C76
:07422400F571C21DF56F22C8
:1040D100EF24FCF55CD3940D4010200B077E377F55
:1040E100D41231C6E4F55CD21A2290744463A20161
:1040F10090787463A201AF5C1224D9C21A200B0D0F
:0E4101007E377FDD7C747D44AB5C122ED222B3
:0F42FB00D3EF6480948D5006E57170028F7122AD
:101B750020D903021C79201C03021C79E5716067DA
:101B85009070CF540FFF7D5E1224D0E55E64017026
:101B95003A9070DEE0B4FF0ED21E200B127E377F26
:101BA500E41231C68009301E06E4F571021C791273
:101BB50041AE123E23200B0D7E377FF27C707DCF28
:101BC500AB71122ED2E4F571021C791241AE123EB0
:101BD50023200B0D7E377FFD7C707DCFAB71122EE0
:101BE500D2E4F571021C79E55C6055907878E024C3
:101BF50005F526D3940D4007E4F55CD21A8075905F
:101C05007874E526540FFF7D5E1224D0E55E30E73B
:101C150002D21DE55E6401701A301E17E561B4013C
:101C250012200B127E387F0A7C707DCFAB71122E8D
:101C3500D28003123E231241AEE4F55CD21A803401
:101C4500E56E601E907758540FFF7D5E1224D0E537
:101C55005EB40103201E03123E231241AEE4F56E6D
:101C65008012201F0C90776CE0C3946450031234EB
:101C7500591241AE122C4D8F26EF7003021D93129F
:101C8500408AE4F56FE55EB4010CD21E200B077E99
:101C9500387F141231C6E570C394C8501B30031841
:101CA500746D2570F582E43477F583E5262570F5A6
:101CB500707D5EAF261224C7300121E55E20E71C4A
:101CC5009076447D5EAF261224C7AF261235D1EF3C
:101CD500700A200B077E387F221231C6E55E5481DB
:101CE5006003021D93E526D3940D4010300B0302CB
:101CF5001D937E387F311231C6021D93E560D39462
:101D050007401F300B03021D939071D07D5EAF26F7
:101D15001224C77E387F3F7C717DD0AB26122ED230
:101D2500806CE50F30E66290789FE0FF903EB493BB
:101D3500FE547F655E7052EFA3936560704B90789B
:101D45009FE0C313FF2486F582E43478F583E070C1
:101D550038530F3F90789FE0FD7471250FF582E4AD
:101D65003461F583EEF0ED903EB593FE7472250F68
:101D7500F582E43461F583EEF074862FF582E43460
:101D850078F5837401F0430F40AF26122DA8300E6D
:101D95001A30001590776CE0C39464500C056FE51C
:101DA5006F94F04004C2AF80FEC20E200203021EF3
:101DB500A8E56D6031D394014004156D80289078B5
:101DC50084E004F0E0D39403400D200B077E387FB8
:101DD5004B1231C6124204200B077E387F58123150
:101DE500C6E4F56DD21C301B43E56E703F90775805
:101DF50004F0A37408F0A37480F0A37401F0A37435
:101E050006F090786FE090775DF0907870E09077CD
:101E15005EF0907871E090775FF0907872E090775F
:101E250060F0E4A3F0A3F0756E0BC21B301972903D
:101E3500786DE07035E56E70319077587442F0A397
:101E45007408F090786EE090775AF0907873E0908F
:101E5500775BF0A37401F0756E06200B077E387F63
:101E6500671231C690786DE004F090786DE06402F9
:101E7500702FE56E702B9077587402F0A37408F0FC
:101E850090786EE090775AF0A3F0A37401F0756E28
:101E950006200B077E387F6E1231C690786DE00400
:081EA500F0C202121EAEC200E1
:011EAD002212
:10417B00E570602CE4907540F0A3E570F090774506
:10418B00E0907542F0A37419F090776D63A20190E3
:10419B00754463A201AF701224D9E4F5707F01223C
:0341AB007F002270
:0B430A00301A05C21A7F01227F00223A
:0100210022BC
:06432F00E4F570F55C22CC
:0A431500E49071D0F0A3F0A3F022B1
:103E85002043616E457247495400200A004572720D
:103E95004C656E43616E21000A002043616E4572D8
:103EA50072434821000A205265714572722100C48F
:103EB50000C401C402C403C404C405C406C407C8BD
:103EC50000C801C802C803C804C805C806C807C297
:103ED50000C201C202C203C204C205C206C2070073
:013EE50000DC
:102C4D00E59B541F6020200B1A7E3E7F851231C6F6
:102C5D00E59B541FFF7E007D031232AE7E3E7F8FBB
:102C6D001231C6E4F59BE5BA30E010E4F5B375B169
:102C7D0080F5B2D21CF56D907884F0E5CFF4700339
:102C8D00022DA5752801E4F527E5CFF4552870032D
:102C9D00022D93E527C454F0F5B1E5B2547F6420BD
:102CAD006003022D64E5B3540FF56285BC5EE5BD8E
:102CBD00541FFF131313541FFFE5BD54E044184F69
:102CCD00F55FE5BDC43354E0FFE5BE131313541F88
:102CDD004FF560E5BEC43354E0FFE5BF1313135445
:102CED001F4FF56185A36385A36485A36585A366E1
:102CFD0085A36785A36885A36985A36AE4F5B220DA
:102D0D001F0FE55E547EB55E0843BDF875B3508068
:102D1D000375B3D0E562700AE55E547EB55E037F40
:102D2D000022301F08E55E30E7037F0022E562D305
:102D3D009408401D200B177E3E7F921231C6AF6264
:102D4D007E007D031232AE7E3E7F9D1231C67F0026
:102D5D0022E5622405FF22E5B2549F6023200B205B
:102D6D007E3E7F9F1231C6AFB27E007D031232AE22
:102D7D00AFB37E007D031232AE7E3E7F9D1231C613
:102D8D00E4F5B275B3D0E52825E0F5280527E5274C
:0A2D9D00C394085003022C967F0037
:012DA7002209
:103E230090776CE0C39464505675B180E4F5B3F5B4
:103E3300B2855EBCE560C4135407FFE55F54E04FF1
:103E4300F5BDE56033333354F8FFE561C41354071C
:103E53004FF5BEE56133333354F8F5BF8563A3856E
:103E630064A38565A38566A38567A38568A3856920
:103E7300A3856AA3E562540F2450F5B3756D0AC296
:023E83001C22FF
:1034590075B190E5B220E613200B107E3E7FAA12CB
:1034690031C6AFB27E007D031232AEE4F5B3F5B2D8
:103479007471250FF582E43461F583E0701B90784F
:103489009FE0FFC3132486F582E43478F583E07066
:1034990005430F808003430F40E50F30E615E4F53F
:1034A9000F90789FE02402F0E0903EB4937004906E
:1034B900789FF0E50F30E72190789FE0FF903EB4C8
:1034C90093F5BCE4F5BDEFA393FF33333354F8F51B
:1034D900BE75BF78430F4080367471250FF582E4BD
:1034E9003461F583E0F5BCE4F5BD7472250FF5820E
:1034F900E43461F583E0FF33333354F8F5BE75BF27
:1035090078050F050FE50FC394324003E4F50F75F5
:03351900B350228A
:09431F00EF6003C29622D296223F
:103C2D0043AB01C2E8C2EAE4FFEFC454F0F5B1C3FF
:103C3D00EF64809488500575B3D08003E4F5B3E448
:103C4D00F5B2F5BCF5BDF5BEF5BFF5C4F5C5F5C6C8
:103C5D00F5C7F5A3F5A3F5A3F5A3F5A3F5A3F5A373
:103C6D00F5A30FBF0EC390776CE0FE25E0F5B4759C
:103C7D00B50C75B66C75A11275AB0275C13E75C3E9
:103C8D00FF75C203E490789FF0750F80FF7F199048
:103C9D007886E4F0A3DFFCE4FF7F32906171E4F0FD
:033CAD00A3DFFC96
:013CB00022F1
:1013A2003E2A2C312CCFE0F0E0ECE5F2F0FB20F30A
:1013B200EFF0E0E2EBFFFEF9E5E3EE20EAEEEDF21C
:1013C200F0EEEBEBE5F0E020CACF20C8F1E5F2FC4D
:1013D2000A003E4C2C6B30312C25732C43EAEEF084
:1013E200EEF1F2FC20EDE020F8E8EDE52043414E7D
:1013F2002C30202D20353030EAE1283530EC292CF4
:1014020031202D203530EAE128353030EC290A0030
:1014120030202D20353030EAE1283530EC290031FA
:10142200202D203530EAE128353030EC29003E42CB
:101432002C6330312C2562752CC2F2EEF0E8F7ED08
:10144200FBE920EAEEEDF2F0EEEBEBE5F020EDE069
:1014520020F8E8EDE50A003E2A2C312CCFF0EEF21E
:10146200EEEAEEEB20C8F1E5F2FC2DCCE0E3E8F188
:10147200F2F0E0EBFCEDFBE920EDE020EFEEF0F224
:10148200F32052533233320A003E4C2C6B30352C4F
:10149200256C752CD1EAEEF0EEF1F2FC20EEE1ECD7
:1014A200E5EDE020EDE020EFEEF0F2F32C3130300C
:1014B2002C3230302C3330302C3630302C3132302C
:1014C200302C323430302C343830302C3936303005
:1014D2002C31393230302C33383430302C353736E9
:1014E20030302C3131353230300A003E532C6B30E3
:1014F200362C2562752CC0E4F0E5F120CACF20E439
:10150200EBFF20ECE0E3E8F1F2F0E0EBE80A003E6A
:10151200532C6B31332C2562752CC7E0E4E5F0E6E1
:10152200EAE020F1F2E0F0F2E020EFE5F0E5E4E0BD
:10153200F7E828E1E0E9F2290A003E422C6B31305B
:101542002C2562752CCFE5F0E5E7E0E3F0F3E7EA5E
:10155200E020EFF0E820EEF2F1F3F2F1F2E2E8E857
:1015620020EEE1ECE5EDE0203220ECE8ED2E0A0081
:101572003C21003C6B30313D003C6330313D003C4E
:101582006B30353D003C6B30363D003C6B31333DBA
:10159200003C6B30393D003C6B31303D00545520EE
:1015A2005265710A005455204F4B0A00CEF820E4D0
:1015B200EBE8EDFB210A000A4173796E634F555443
:1015C2003A002054552054696D65210A000A43529D
:1015D20043204552523A20000A4173796E63494EC4
:1015E2003A00CFE0EAE5F220E22043414E0A000A47
:1015F200CFF0E8EDFFF2E020EAEEECE0EDE4E020EF
:10160200D2D320002020D2D320E7E0EDFFF2EE215A
:101612000A003F3F3F0A000089129B24AD36BF48B3
:10162200C15AD36CE57EF78108931AA52CB73EC93F
:1016320040DB52ED64FF76028B109926AF34BD4A2F
:10164200C358D16EE77CF5830A9118A72EB53CCB1F
:1016520042D950EF66FD74048D169F20A932BB4C0F
:10166200C55ED768E17AF3850C971EA128B33ACDFF
:1016720044DF56E960FB72068F149D22AB30B94EEF
:10168200C75CD56AE378F1870E951CA32AB138CFDF
:1016920046DD54EB62F97008811A932CA53EB740DF
:1016A200C952DB64ED76FF89009B12AD24BF36C1BF
:1016B20048D35AE56CF77E0A8318912EA73CB542AF
:1016C200CB50D966EF74FD8B029910AF26BD34C39F
:1016D2004AD158E76EF57C0C851E9728A13AB3448F
:1016E200CD56DF60E972FB8D049F16A920BB32C57F
:1016F2004CD75EE168F37A0E871C952AA338B1466F
:10170200CF54DD62EB70F98F069D14AB22B930C75E
:101712004ED55CE36AF17800112332465765748C2A
:101722009DAFBECADBE9F810013322564775649CAF
:101732008DBFAEDACBF9E82130021367764455AD9E
:10174200BC8E9FEBFAC8D93120120377665445BD8F
:10175200AC9E8FFBEAD8C94253617004152736CE7E
:10176200DFEDFC8899ABBA5243716014053726DE6F
:10177200CFFDEC9889BBAA6372405125340617EF5E
:10178200FECCDDA9B88A9B7362504135241607FF4F
:10179200EEDCCDB9A89A8B8495A7B6C2D3E1F00846
:1017A200192B3A4E5F6D7C9485B7A6D2C3F1E0182F
:1017B200093B2A5E4F7D6CA5B48697E3F2C0D1291E
:1017C200380A1B6F7E4C5DB5A49687F3E2D0C1390F
:1017D200281A0B7F6E5C4DC6D7E5F48091A3B24AFE
:1017E2005B69780C1D2F3ED6C7F5E49081B3A25AEF
:1017F2004B79681C0D3F2EE7F6C4D5A1B082936BDE
:101802007A48592D3C0E1FF7E6D4C5B1A092837BCE
:071812006A58493D2C1E0F2E
:0300230002351C87
:0D351C00C0E0C0F0C083C082C0D075D018E0
:1035290030985AC298750B01AF99202013BF5509DD
:10353900754D00D220D2918044906B88EFF0803D88
:10354900E55670347489254DF582E4346BF583EFC3
:10355900F0E54DB40104EF04F546E54D600AB546C2
:103569001304F556C291800CEF64556007C2209090
:103579006B88EFF0054D8005906B88EFF030993D31
:10358900302138D290E554700DE54A654960070548
:103599004A75990A8025E554B54C10C221754A002F
:1035A900D223C290E4FF12431F801074892554F579
:0D35B90082E4346CF583E0F5990554C29965
:0B35C600D0D0D082D083D0F0D0E03213
:10372F007BFF7A1379A212187B90776CE070147577
:10373F002EFF752F147530127BFF7A1379D4121860
:10374F007B8012752EFF752F147530217BFF7A1336
:10375F0079D412187B7BFF7A147930A21FE433F5EA
:10376F002E12187B7BFF7A14795912187B9070C92F
:10377F00E0FEA3E0FFC3E49FFFE49EFEAB07FA3336
:10378F0095E0F9F87F007E8C7D0A7C001221BD8FB9
:10379F00318E308D2F8C2E7BFF7A14798B12187B04
:1037AF007BFF7A1479ED85552E12187B7BFF7A15E6
:1037BF00791185492E12187B7BFF7A15793C855735
:0537CF002E12187B2200
:1030DD007E157F72123A9FEF4E70037F0122E490AE
:1030ED00776CF07E157F75123A9FEF4E6015124288
:1030FD00D1BF310690776C740AF0BF320690776CB1
:10310D007464F07E157F7B123A9FEF4E600D123E78
:10311D00E6EC4D4E4F24FF921F8002C21F7E157F9D
:10312D0081123A9FEF4E6023123EE6A804A905AA2C
:10313D0006AB077F007E8C7D0A7C001221BD12221A
:10314D004F9070C9EEF0A3EFF0800A9070C974FF34
:10315D00F0A374B8F07E157F87123A9FEF4E60078B
:10316D00123EE68F558003755501906B867401F004
:10317D007E157F8D123A9FEF4E6007123EE68F4906
:10318D008003E4F5497E157F93123A9FEF4E600C54
:10319D001242D1EF24D024FF92228002D2227E153A
:1031AD007F99123A9FEF4E600A1242D1EF24D0F56B
:0831BD00578003E4F5577F0081
:0131C50022E7
:10368100C221C223C220E4906B87F0F554F54CF5BA
:10369100089061A4F0F54DF50BF54A9070C974FFDF
:1036A100F0A374F4F01230DDE4F50FF558E5587528
:1036B100F00DA42403F582E43461F583E4F0F54BC5
:1036C10075F068E558A42489F582E5F0346DF58339
:1036D10075F00DE54B1222ABE4F0054BE54BB40858
:1036E100DF0558E558B408C5E4F55BF544F545F543
:1036F10047F553F558F54BF552C2ADF5C9D2CDD2C8
:10370100CCC2C9C2CAF5CDF5CC9070C9E0F5CBA346
:10371100E0F5CA85CBCD85CACCD29ED29CD2CAC295
:0E372100ACC298C29975B81075B710D2AC2220
:0100220022BB
:102DA8008F27E55EB44209E56164027003022ED103
:102DB800E55F54E324DF607824DF7003022E8D146E
:102DC8007003022EA124E37003022E601470030224
:102DD8002E6024E1601E24606003022ED1E5607538
:102DE800F00DA42403F582E43461F5837D5EAF27FA
:102DF8001224C722E56075F00DA42403F582E4349B
:102E080061F583E4F075F00DE547A42446F582E505
:102E1800F03468F5837D5EAF271224C70547534712
:102E28003FE54565476003022ED1054553453F22DE
:102E380075F00DE544A424C5F582E5F03461F58309
:102E48007D5EAF271224C7054453447FE544655B84
:102E58007077055B535B7F22435F0143618075F0A8
:102E680068E560A42489F582E5F0346DF583E561B1
:102E7800543FFF1313543F75F00D1222AB7D5E7F54
:102E88000D1224C722300C077E157F9F1231C630E1
:102E9800193790786D7402F022300C077E157FA7E1
:102EA8001231C675F00DE547A42446F582E5F034E5
:102EB80068F5837D5EAF271224C7054753473FE572
:0A2EC80045B54705054553453F2277
:103FF8008E2A8F2B8F828E83E5822404F582E43506
:1040080083F583E02405F554D3940E400B200B2A46
:104018007E157FAE1231C622852A83852B8263A244
:104028000174892552F582E4346CF58363A201AFEB
:0B403800541224D9E5542552F5522201
:1025E700E4F529755206F528906B86E0FFE529C3C7
:1025F7009F4003022721E5476545601E75F00DE5FD
:1026070045A42446F582E5F03468AF82FE123FF810
:10261700054553453F0529022715E54814602E1443
:1026270060728000E4F548E544655B601E75F00D57
:10263700E55BA424C5F582E5F03461AF82FE123F65
:10264700F8055B535B7F05290227150548E5537598
:10265700F00DA42403F582E43461F583E0602EE5F0
:102667005375F00DA42403F582E43461AF82FE12A2
:102677003FF8E55375F00DA42403F582E43461F5C2
:1026870083E4F005535353070529022715055353D0
:102697005307054875F068E558A42489F582E5F0E5
:1026A700346DF58375F00DE54B1222ABE0604C7588
:1026B700F068E558A42489F582E5F0346DF5837553
:1026C700F00DE54B1222ABAF82AE83123FF875F0E7
:1026D70068E558A42489F582E5F0346DF58375F033
:1026E7000DE54B1222ABE4F0E54BC394084008E438
:1026F700F54B055853580705298013054BE54BC380
:1027070094084008E4F54B05585358070548052831
:10271700E528C3940A50030225EFE55224FAF52968
:10272700906C897455F0A3F0E5292405A3F0E4A380
:10273700F0A3E555F0906845E0906C8EF0E4F54E17
:10274700F54FE5292403F551906C8C63A20190168F
:102757001963A201AF51AE50AD4FAC4E1225158F84
:10276700518E508D4F8C4E748F2529F582E4346C31
:10277700F583E54FF074902529F582E4346CF583F1
:10278700E54EF0E5292408F54CD221E4F554906193
:102797006FF07F0112431FD299200B0D7E157FB971
:0927A7007C6C7D89AB4C122ED232
:0127B0002206
:101EAE00E55375F00DA42403F582E43461F583E067
:101EBE007005055353530775F068E558A42489F54A
:101ECE0082E5F0346DF58375F00DE54B1222ABE033
:101EDE007011054BE54BC394084008E4F54B0558CB
:101EEE00535807300034C20030191890616EE00468
:101EFE00F0E0D3940A400C200B077E157FC41231FC
:101F0E00C6C219E557600D0557E557D394F0400446
:101F1E00C2AF80FE90616FE004F030DA3FC2DA901B
:101F2E0061A4E0FF906B87E0FDC39F502FE55A251B
:101F3E00ECF5EC30D709E55925FC04F5FC8006E5F7
:101F4E005925FCF5FC74A52DF582E43461F583E08A
:101F5E00B555031225E7906B87E004F030210F9002
:101F6E00616FE0D39414400BC221D2238005E4901C
:101F7E00616FF0906B88E0FF600C7E007D03123283
:101F8E00AEE4906B88F0E5567003022180F527E4ED
:101F9E00F54EF54FE52724FEF551906B8B63A201AC
:101FAE0090161963A201AF51AE50AD4FAC4E122533
:101FBE00158F518E508D4F8C4EC220E4F556E54F45
:101FCE00454E601D300B030221807E157FCF7C6B4A
:101FDE007D89AB27122ED27D03AF4FAE4E1232AE9D
:101FEE0022200B0D7E157FDA7C6B7D89AB27122E9E
:101FFE00D2906B8BE0FB640160030220EB906B8D43
:10200E00E09061A3F06007E020E703022180906179
:10201E00A3E0547FF0906845F0E5E92402F5EC303A
:10202E00D707E5F904F5FC800385F9FCC2DA906B5D
:10203E008CE075F064A485F059F55A906B8EE0FE35
:10204E00541F9061A4F0EEC413540704906B86F0F5
:10205E00E4A3F0F5279061A4E0FFE527C39F501E8F
:10206E00748F2527F582E4346BF583E0FF74A52584
:10207E0027F582E43461F583EFF0052780D7748F5E
:10208E002527F582E4346BF583E0F46003022180AA
:10209E0074912527F582E4346BF583E0FF90787018
:1020AE00E06F700302218074902527F582E4346B73
:1020BE00F583E090786FF0A3EFF074922527F58208
:1020CE00E4346BF583E0907871F074932527F582F4
:1020DE00E4346BF583E0907872F0D21B22906B8C17
:1020EE00E065556003022180EB24FD6038047078B2
:1020FE00200B077E157FE41231C6E56E7074756E87
:10210E000D906B8E63A20190775863A201AF6E1291
:10211E0024D9907758E06444705890775DE07052FF
:10212E00F545F54722200B077E157FF11231C6309B
:10213E00190B200B3D7E167F061231C622906B8F37
:10214E00E090786EF0906B90E025E0907873F090D0
:10215E006B91E020E006907873E004F0D219E490E1
:10216E00616EF090786DF022200B077E167F1412B0
:02217E0031C668
:01218000223C
:10391100020885E493A3F8E493A34003F68001F23F
:1039210008DFF48029E493A3F85407240CC8C333B7
:10393100C4540F4420C8834004F456800146F6DF86
:10394100E4800B0102040810204080904328E47EAB
:10395100019360BCA3FF543F30E509541FFEE4937B
:10396100A360010ECF54C025E060A840B8E493A342
:10397100FAE493A3F8E493A3C8C582C8CAC583CA6D
:10398100F0A3C8C582C8CAC583CADFE9DEE780BE25
:01432E00008E
:1021810075F008758200EF2FFFEE33FECD33CDCC15
:1021910033CCC58233C5829BED9AEC99E582984098
:1021A1000CF582EE9BFEED9AFDEC99FC0FD5F0D675
:1021B100E4CEFBE4CDFAE4CCF9A88222B800C1B99F
:1021C1000059BA002DEC8BF084CFCECDFCE5F0CBDD
:1021D100F97818EF2FFFEE33FEED33FDEC33FCEB16
:1021E10033FB10D703994004EB99FB0FD8E5E4F9D1
:1021F100FA227818EF2FFFEE33FEED33FDEC33FCBE
:10220100C933C910D7059BE99A4007EC9BFCE99AB1
:10221100F90FD8E0E4C9FAE4CCFB2275F010EF2FF6
:10222100FFEE33FEED33FDCC33CCC833C810D707F6
:102231009BEC9AE899400AED9BFDEC9AFCE899F831
:0E2241000FD5F0DAE4CDFBE4CCFAE4C8F922C4
:0E224F00C3E49FFFE49EFEE49DFDE49CFC22A0
:10225D00EB9FF5F0EA9E42F0E99D42F0E89C45F0D7
:01226D00224E
:0C226E00ECF0A3EDF0A3EEF0A3EFF022E3
:10227A00A8828583F0D083D08212229112229112F1
:10228A002291122291E473E493A3C583C5F0C58316
:10229A00C8C582C8F0A3C583C5F0C583C8C582C8AE
:0122AA002211
:0C22AB00A42582F582E5F03583F583223E
:10181900E53A242EF8E6053A22782B301702782E7D
:10182900E475F00112235E0222B72010EB7F2ED25D
:10183900108018EF540F2490D43440D4FF30140B87
:10184900EF24BFB41A0050032461FFE53B60021581
:101859003B053EE53E7002053D30170D782BE475DA
:10186900F00112235EEF0222FD0240437403D217F6
:101879008003E4C217F53A8B2B8A2C892DE4F53BBA
:10188900F53DF53EE53B60077F2012185480F5755C
:101899003CFFC211C210C212C213C215C216C2182D
:1018A900121822FF700D3017057F00121865AF3E20
:1018B900AE3D22B4255FC2D5C214121822FF24D02E
:1018C900B40A00501A75F00A783B30D50508B6FFFE
:1018D9000106C6A426F620D5047002D21380D924A5
:1018E900CFB41A00EF5004C2E5D214021A65D2111E
:1018F90080C6D21080C0D21280BCD2D580BAD2158F
:1019090080B47F201218542012077401B53B00409F
:10191900F1121819FF12185402188DD218D2168014
:1019290095121819FB121819FA121819F94A4B705D
:101939000679367A1B7BFF20122EE53B602A7E0052
:101949008E827583001222D060060EEE653C70F01F
:10195900C2D5EBC0E0EAC0E0E9C0E0EE121AACD0B3
:10196900E0F9D0E0FAD0E0FB1222B7FF60AAEBC0A1
:10197900E0EAC0E0E9C0E0121854D0E02401F9D04F
:10198900E03400FAD0E0FBE53C0460DCD53CD980CA
:10199900877BFF7A1A79A8D212809C791080027904
:1019A90008C216C2188008D2D5790A8004790AC2F9
:1019B900D5E53C047002F53CE4FAFDFEFF12181966
:1019C900FC7B08201113121819FD7B1030100A1224
:1019D9001819FE121819FF7B20EC3382D592D550C5
:1019E90013C3E43010069FFFE49EFEE42011039D1B
:1019F900FDE49CFCE4CBF8C211EC700CCFCECDCC4D
:101A0900E824F8F870F38017C3EF33FFEE33FEEDE7
:101A190033FDEC33FCEB33FB994002FB0FD8E9EBC8
:101A2900301105F8D0E0C448B211C0E00AEC4D4EBF
:101A39004F78207B0070C2EAB53C0040BCC0E01280
:101A49001AAED0F0D0E0201104C4C0E0C4B211C075
:101A5900F012183DD0F0D5F0EB02188D1223BD1904
:101A69002A5319A45818FB4C18F74219A84F19B052
:0F1A79004419B04919104319B655199A46199ACC
:101A880045199A471B565018FF2D19032E19262B56
:101A98001907231924201B3F2A18BF480000191EC4
:101AA8003F3F3F00790AA2D5201314301509B91019
:101AB800020404B9080104A2D5201602500104202A
:101AC80012689212B53B005034C0E07F20301319E1
:101AD8007F30A21272167215500F121B05C212C265
:101AE80016C215C2187F30800F301503E9C0E01206
:101AF8001854301503D0E0F9D0E0B53BCC301517B9
:101B08007F30B9100C1218547F583014077F788032
:101B180003B908031218543012057F2D0218547F98
:101B2800202018F87F2B2016F322921280CF286EDF
:101B3800756C6C2900D2111218193011F8C211787D
:101B48003B30D50108F60218BF2D504349581218EA
:101B5800192403B405004001E4901B519312184561
:0D1B6800743A121845D213753B040219A4FB
:1027B1008B268A278928E4F532F531F530F52FF596
:1027C1002DF52EE52A452B45296012EBC0E0EAC024
:1027D100E0E9C0E0AB29AA2AA92B12236EAB26059A
:1027E10028E528AA277002052714F91222B7F53324
:1027F100C394094007E533D3940D40E1E5336420E8
:1028010060DBE533B42D05432E038016E533B42B8D
:1028110005432E01800C74FF2528F52874FF352708
:10282100F527E52C60046410703FAB26AA27A92880
:102831001222B764306009E52C702E752C0A8029AC
:102841009000011222D0FF64786004EFB458134362
:102851002E01752C1074022528F528E43527F5275B
:102861008007E52C7003752C08AB260528E528AAFE
:10287100277002052714F91222B7F533C39461407A
:102881000AE533D3947A50035333DF74D02533F5FB
:1028910033C3940A400CE5339411406D74F9253328
:1028A100F533E533D3952C5060432E0185323785BE
:1028B1003136853035852F34AF2C7E00E4FCFDABFD
:1028C10032AA31A930A82F12230FC8ECC8C9EDC90B
:1028D100CAEECACBEFCBE4FCFDFEEB2533F532EEBD
:1028E1003AF531ED39F530EC38F52FAF32AE31AD87
:1028F10030FCAB37AA36A935A834D312225D500378
:1029010002286A432E0402286AE52E20E003E480AF
:102911002DE52A452B4529601EAB26E52824FFF924
:10292100E52734FFFAEBC0E0EAC0E0E9C0E0AB29FB
:10293100AA2AA92B12236EE52E30E20774FFFFFEAF
:10294100FDFC22E52EAF32AE31AD30AC2F30E103CC
:0429510002224F22ED
:1022B700BB010689828A83E0225002E722BBFE0225
:0922C700E32289828A83E4932258
:1022D000BB010CE58229F582E5833AF583E02250C3
:1022E00006E92582F8E622BBFE06E92582F8E2220D
:0D22F000E58229F582E5833AF583E4932227
:1022FD00BB010689828A83F0225002F722BBFE01C0
:02230D00F322B9
:10230F00E88FF0A4CC8BF0A42CFCE98EF0A42CFC6D
:10231F008AF0EDA42CFCEA8EF0A4CDA8F08BF0A4EB
:10232F002DCC3825F0FDE98FF0A42CCD35F0FCEB4A
:10233F008EF0A4FEA9F0EB8FF0A4CFC5F02ECD390F
:0F234F00FEE43CFCEAA42DCE35F0FDE43CFC227C
:10235E00FAE6FB0808E6F925F0F618E6CA3AF62280
:10236E00BB011A89828A83D0F0D0E0F8D0E0F9D090
:10237E00E0FAD0E0FBE8C0E0C0F00223EC5016E932
:10238E00F8D083D082D0E0F9D0E0FAD0E0FBC08262
:10239E00C0830223E3BBFE16E9F8D083D082D0E0DF
:0F23AE00F9D0E0FAD0E0FBC082C0830223F52211
:1023BD00D083D082F8E4937012740193700DA3A3AF
:1023CD0093F8740193F5828883E4737402936860C3
:0623DD00EFA3A3A380DFC3
:0923E300EBF608EAF608E9F6221F
:0923EC00EBF0A3EAF0A3E9F022F2
:0923F500EBF208EAF208E9F22219
:00000001FF
